:100000000C9450010C9479010C9479010C947901B1
:100010000C9479010C9479010C9479010C94CE0222
:100020000C9479010C9479010C9479010C94790168
:100030000C9479010C9479010C9479010C94790158
:100040000C9479010C9479010C947C030C94790143
:100050000C9439030C9479010C9479010C94790176
:100060000C9479010C947901437934436F6465A051
:10007000027013B0012020F0FF000100025F0200B7
:10008000FFFF003D0002290240FFFF0001000114B4
:1000900002F0FFFF00070000E901F8FFFF00010088
:1000A00001D601FAFFFF00010001C301FCFFFF00C0
:1000B0000200017B0120620501806A060101110630
:1000C000010000000002000002000000010000002A
:1000D0000100000001020C06030000000200000005
:1000E000020000000220620501406205010464066E
:1000F000040000000310350603080C060000000091
:100100000400000004005EBCE2613FDD83C29C7E0F
:1001100020A3FD1F419DC3217FFCA2401E5F01E380
:10012000BD3E6082DC237D9FC1421CFEA0E1BF5D1D
:100130000380DE3C62BEE0025CDF81633D7C22C066
:100140009E1D43A1FF4618FAA427799BC584DA387F
:1001500066E5BB5907DB856739BAE406581947A538
:10016000FB7826C49A653BD987045AB8E6A7F91BE1
:1001700045C6987A24F8A6441A99C7257B3A64861E
:10018000D85B05E7B98CD2306EEDB3510F4E10F24B
:10019000AC2F7193CD114FADF3702ECC92D38D6FE8
:1001A00031B2EC0E50AFF1134DCE90722C6D33D1B5
:1001B0008F0C52B0EE326C8ED0530DEFB1F0AE4CCE
:1001C0001291CF2D73CA947628ABF517490856B40F
:1001D000EA6937D58B5709EBB536688AD495CB29B0
:1001E00077F4AA4816E9B7550B88D6346A2B759769
:1001F000C94A14F6A8742AC896154BA9F7B6E80A96
:1002000054D7896B35020403050606070708080959
:100210000901590601000000000000000000000074
:1002200000200000000200000200000001000000A9
:1002300001020000030000000200000002000000B4
:10024000024000000020000000800000000455066D
:100250000410310603080000000000000400000044
:1002600004015B4379344E75742042617369635DA8
:10027000000000000000000000000000000000007E
:10028000000000000000000000000000000000006E
:10029000000000000000000000000000000000005E
:1002A00011241FBECFEFD8E0DEBFCDBF14BE0FB606
:1002B000F894A89580916000886180936000109206
:1002C00060000FBE11E0A0E0B1E0ECE8F9E102C08F
:1002D00005900D92A830B107D9F723E0A8E0B1E06E
:1002E00001C01D92AD35B207E1F70E94F40A0C94EB
:1002F000C40C0C940000EF92FF920F931F93CF93C6
:10030000DF9300D000D0CDB7DEB77C018B010E9417
:100310007D0A9A838983CE0101960E940D058B8305
:10032000CE0101960E9410058C83AE014D5F5F4F98
:10033000B801C7010E94C80A8B8189838C818A8396
:10034000CE0101960E942105882321F0C8010E9458
:100350002E050EC0CE0101960E9413058823B1F32D
:1003600089819A810E947B0ACE0101960E94630BCB
:100370000F900F900F900F90DF91CF911F910F91E1
:10038000FF90EF900895CF93DF93EB01CB010E9494
:100390004005FC0180818E3521F4DF91CF910C94D2
:1003A000C303CE01DF91CF910C942E05CF93DF9341
:1003B000EB01CB010E944005FC0180818E3521F4C8
:1003C000DF91CF910C94C003CE01DF91CF910C94BB
:1003D0002E05FF920F931F93CF93DF93EC018B01B8
:1003E000CB010E943705F62ECE010E94C20AF61AF2
:1003F000D0E0CD2FCF0DC8010E943D05D81770F475
:10040000C8010E944205EC2FF0E0E159FF4FE49152
:10041000DC01AD0FB11DEC93DF5FEBCFDF91CF912E
:100420001F910F91FF900895CF93DF93EB01CB01C4
:100430000E944005FC0180818E3531F40E941A0B28
:10044000DF91CF910C94C003CE01DF91CF910C943A
:100450002E05EF92FF920F931F93CF93DF93CDB7AB
:10046000DEB7ED970FB6F894DEBF0FBECDBF8C019F
:100470007B014DE350E0BE016F5F7F4F8BE090E06A
:100480000E94110BAE014F5F5F4FB701C8010E9480
:10049000C80A1DAE4DE350E06BE070E0CE0101965E
:1004A0000E94130BED960FB6F894DEBF0FBECDBFC2
:1004B000DF91CF911F910F91FF90EF9008950F93CF
:1004C0001F93CF93DF931F92CDB7DEB78B01CB0184
:1004D0000E943405811110C041E050E0BE016F5F01
:1004E0007F4F8AE090E00E94110BC8010E944205F4
:1004F0002981FC01208315C0C8010E944005FC0130
:1005000091E08081811101C090E0998341E050E049
:100510006AE070E0CE0101960E94130B89810E946F
:100520008B040F90DF91CF911F910F910895CF937E
:10053000DF931F92CDB7DEB786E790E00E945F0A97
:100540000E943E0B0E947B0A41E050E0BE016F5FBB
:100550007F4F8AE090E00E94110B89810E948B04FA
:100560000F90DF91CF91089508950895F89498E041
:1005700088E10FB6F894A895809360000FBE909321
:100580006000E0E0F1E080E099E08193E030F9077D
:10059000E0F3FFCF87FF01C0789408951F920F9278
:1005A0000FB60F9211242F938F939F93EF93FF9386
:1005B00080910A01843021F410920A018BE204C078
:1005C0008F5F80930A018AE28093B30080912802B2
:1005D000909129020196909329028093280280919C
:1005E0000801909109010196883E23E0920729F0C5
:1005F00090930901809308010DC010920901109297
:10060000080180912602909127020196909327027B
:10061000809326028091D70186958695869590E0F5
:100620000497ECF48091D701887F98E0980F80912F
:10063000D7018770892B8093D7018091D701869548
:100640008695869590E0049754F0E0910D01F0E0D6
:10065000EE0FFF1FE15FFE4F808181608083FF917D
:10066000EF919F918F912F910F900FBE0F901F9040
:1006700018951F920F920FB60F9211248F939F938C
:10068000EF93FF938091D70181FD07C08091D7013F
:1006900084608093D7011092D9018091D7018D7F1A
:1006A0008093D7018091DA019091D901911106C010
:1006B0009091D7019E7F9093D70113C0E82FF0E06F
:1006C000E552FE4F90819093D80190819093C6009F
:1006D0008F5F8B3409F480E09091D9019150909311
:1006E000D9018093DA01FF91EF919F918F910F9043
:1006F0000FBE0F901F9018951F920F920FB60F927A
:1007000011248F939F93EF93FF939091C600809154
:10071000D70187708093D7018091D70180FF09C0EE
:100720008091D801981305C08091D7018260809391
:10073000D70180910D01E82FF0E0EE0FFF1FE15F80
:10074000FE4F91838F5F843609F480E090910E0113
:1007500089130BC0E0910D01F0E0EE0FFF1FE15F88
:10076000FE4F80818160808302C080930D01FF91E4
:10077000EF919F918F910F900FBE0F901F90189542
:1007800010920C01089581E080930C010895CF939D
:10079000DF938FB7F894C0912802D09129020E946C
:1007A000CA02CE01DF91CF9108959C01CB01B9011E
:1007B0000C94920C0C94A20CCF938FB7F894909158
:1007C000D70190FD0AC02091D70126952695269540
:1007D00030E0C1E0243031050CF4C0E00E94CA02D0
:1007E0008C2F8170CF910895CF93DF93C82F8FB74F
:1007F000F894D091D9010E94CA02DB34C1F38FB7BB
:10080000F8949091D70192FD24C09091D70190FF68
:1008100012C0E091DA019091D901E90FEB3408F0B0
:10082000EB54F0E0E552FE4FC0839091D9019F5FF9
:100830009093D9010EC09091D70191609093D70108
:100840009091D7019D7F9093D701C093D801C09319
:10085000C600DF91CF910C94CA02CF938FB7F89462
:10086000C091D701C1700E94CA028C2FCF91089508
:10087000CF938FB7F894C091D701C2FBCC27C0F9B2
:100880009091D7019B7F9093D7010E94CA028C2F31
:10089000CF910895CF93DC018FB7F894C0E0909189
:1008A0000E01E92FF0E0EE0FFF1FE15FFE4F208108
:1008B00020FD0EC020910D01921751F0319620813C
:1008C0002C939F5F943609F490E090930E01C1E061
:1008D0000E94CA028C2FCF910895CF938FB7F894BE
:1008E00090910E01E92FF0E0EE0FFF1FE15FFE4F48
:1008F000C081C17020910D01921719F090819E7FE7
:1009000090830E94CA0281E08C27CF91089589E1EB
:1009100080930B01089580930001811101C05F98BD
:10092000089580910C0181110E94B602F8949FE015
:1009300088E10FB6F894A895809360000FBE90935D
:10094000600087E084B915B88FEC87B918B88CE9D6
:100950008AB91BB88DED90E001970000E9F781EAB4
:1009600084BD83E085BD17BC18BC82E08093B000D5
:1009700096E09093B1002AE22093B3008093700038
:1009800023E230E03093C5002093C4001092C000F1
:1009900028ED2093C1009093C200789480930C01BD
:1009A000089581E090910C01923009F080E0089563
:1009B000A8950E94C70320910001222341F080786E
:1009C00092708038910511F45F9A01C05F98809110
:1009D0000B01882341F0815080930B01882311F093
:1009E000289A0895289808950E942D048111FCCF1B
:1009F00080910C01882361F0813061F4E0E0F8E738
:100A0000859194918C30944929F40C94023C08957A
:100A10000E94B6020895962F0895FC0180810895E2
:100A2000FC0181810895FC0180818F3F39F491E0C0
:100A300081818F3F09F490E0892F01C081E08170AE
:100A40000895FC018081882331F091E0818181113A
:100A500090E0892F01C081E081700895FC0110822F
:100A60000895FC0180810895FC0181810895FC01B5
:100A700064817581868197810895FC018085089540
:100A80000996089509960895DC019BE4EFECF2E0E5
:100A900001900D929A95E1F71092CE020895EDE241
:100AA000F2E0818180958370806C81838281848370
:100AB00083818583A3E0B1E08C91828311968C9130
:100AC000838308950E944F0510922D020895EF929E
:100AD000FF920F931F93CF93DF93DC012C9130E0B3
:100AE0008901E4E0000F111FEA95E1F7A0E0B0E012
:100AF000C0E0D0E0F801EA0FFB1FE40FF51FF4900F
:100B0000FF2061F1FB01E080EF2DEE2111F1220FBA
:100B1000331F220F331F2C0F3D1F220F331F220FB5
:100B2000331FF9013196E40FF51F65917491F901B6
:100B30003396E40FF51FE491DC01EC936115710528
:100B400069F0FB01DF91CF911F910F91FF90EF9022
:100B5000099421961496A031B10561F6DF91CF91E9
:100B60001F910F91FF90EF900895FC01DB0181E050
:100B700090819A3A09F080E08C938181815C91E0C8
:100B8000823008F490E011969C931197848112961C
:100B90008C931297858113968C931397468150E01E
:100BA00060E070E0BA01552744278085480F511D49
:100BB000611D711D878190E0982F8827480F591F6C
:100BC000611D711D14964D935D936D937C931797E2
:100BD000918518969C931897818180FF09C03A9659
:100BE000199680E0891721F021912D938F5FFACF1C
:100BF00008951F93CF93DF93EC01162F0E94C70334
:100C0000810F911D009711F481E090E09983888312
:100C1000DF91CF911F9108956AEF8AE792E00C94DB
:100C2000F9058DE292E00E94440562E388E792E0D4
:100C30000C94F905CF93DF93EC010E94C7038370F6
:100C40009927019690910101890F803108F083E086
:100C50008093010160910101CE01DF91CF910C944D
:100C6000F90588EC92E00C941A0688E792E00C945F
:100C70001A060F931F93CF93DF93FC01218120FF6E
:100C800003C01185155F01C01BE0082FC82FD92FA5
:100C90008C2F801B811720F489910E94F403F8CFD8
:100CA000DF91CF911F910F9108958DE792E00C9401
:100CB00039068DE792E00E9444056AEF8AEC92E0E3
:100CC0000E94F9050C9487048DE292E00E94390697
:100CD0000C9487040E944F0562E388E792E00C942D
:100CE000F905CF92DF92EF92FF920F931F93CF936C
:100CF000DF93EC018B017A0169018091CE02882398
:100D0000B1F18091D00281FF06C08091CC02816058
:100D10008093CC022CC090910201943041F191114A
:100D200024C0817091E0892720912E0221709227A2
:100D30008917D9F085E092E0FC01A4913196E49105
:100D4000B0E0A153BD4FF0E0E35DFD4F3C91208149
:100D500032130BC00296F2E081319F0769F7809150
:100D60007C02816080937C0202C01092CE0280914E
:100D7000CD028430E1F0809102018430C1F00E9404
:100D8000DC038823A1F0F70180819181892B61F038
:100D90000E94C703F70120813181281B390B1216ED
:100DA00013062CF011821082888184608883F801F8
:100DB00080819181892B61F00E94C703F801208115
:100DC0003181281B390B121613062CF01182108268
:100DD000888180628883F2E0CC3CDF07A1F48091B7
:100DE000CD02843009F50E942D0481111DC00E949E
:100DF00038049091CC02882311F0906101C0986072
:100E00009093CC0211C080910201843069F40E9459
:100E10002D04811109C00E9438049881882311F0A3
:100E2000906101C098609883F6018281882331F037
:100E300081E09381992319F080E001C081E080FF77
:100E400003C0888180688883F60180818A3A19F01E
:100E5000888180648883DF91CF911F910F91FF90EB
:100E6000EF90DF90CF9008952DE732E048EC52E00C
:100E70006AEC72E08CEC92E00E94710641E152E073
:100E80006CEC72E08DEC92E00E9467051092CC024F
:100E900008952DE232E048E752E06AE772E08CE71D
:100EA00092E00E94710645EB50E06CE772E082E050
:100EB00091E00E94670510927C020895DF92EF9204
:100EC000FF920F931F93CF93DF93FB011082FC01DE
:100ED0002081222309F48CC0FF24F3942181213046
:100EE00009F4F12CF2E06D327F0709F4F094EB0184
:100EF0008C01FC01328123816D52724091F0DC80C3
:100F0000D31276C0ED80E21273C08A8191E088230B
:100F100019F02B81211190E090FF64C0E12CD12CBD
:100F200061C080910301909104014AEA48834F2DEA
:100F30004370406C49833A832B838C839D83F801F3
:100F400086818E8385818F838481888780858134A3
:100F500010F4898701C01986DE01CE010A96EFEFF1
:100F60002D91E227F0E0EB5FFE4FE491A817B9075F
:100F7000B9F7F0FE19C080E09985891798F4282FF9
:100F800030E0D801A20FB31F19969C91DE01A20F89
:100F9000B31F1A969C93E927F0E0EB5FFE4FE491B4
:100FA0008F5FEACF865F01C08AE0DE01A80FB11D26
:100FB000EC938A81882331F081E09B81992319F099
:100FC00080E001C081E080FF13C08981833C29F467
:100FD0009E81907F81E0903E09F080E080FD08C016
:100FE000188206C06B810E940B053D2D2E2D9DCFD2
:100FF000DF91CF911F910F91FF90EF90DF900895B7
:1010000090930401809303010895809103019091CE
:1010100004010895CF93DF93EC010E942E05809187
:10102000CD02813071F4BE018DE792E00E94B505DA
:101030008091CC0282608093CC020E94340781E0D0
:1010400001C080E0DF91CF9108952091CD02223040
:1010500069F46DE772E00E945E078091CC028260C5
:101060008093CC020E94340781E0089580E00895C7
:1010700020910201223069F46DE272E00E945E0765
:1010800080917C02826080937C020E94490781E00B
:10109000089580E00895CF93DF93EC010E942E0520
:1010A00080910201813071F4BE018DE292E00E94D4
:1010B000B50580917C02826080937C020E94490782
:1010C00081E001C080E0DF91CF91089581E09091AF
:1010D0000201923009F080E008951092CD0282E082
:1010E000809302011092CE02E3E0F1E08FEF808363
:1010F000818308950F931F93CF93DF931F92CDB7F2
:10110000DEB78091CE02811181C00E946D048111F1
:1011100002C010922C021AE00FEFCE0101960E943D
:101120004A04882309F472C090912C02E98191301D
:1011300059F018F0993081F01CC0EA3A71F7109319
:101140002B0200932A0215C08E2F86958695803338
:1011500081F010922C02E1CF8FEF8E0F8034C8F710
:101160008091D00280FF05C080912B028E0F80936A
:101170002B02A92FB0E0A153BD4FEC9380912A021E
:10118000E827F0E0EB5FFE4FE491E0932A028091C4
:101190002B02981337C010922C02E11137C08091B6
:1011A000D10290910301891711F081112FC0909104
:1011B000D20220910401921711F0911127C02091C1
:1011C000D302222319F12091D4022223F9F088239B
:1011D00029F081E0992319F080E001C081E080FFCF
:1011E0000DC08091D002833C31F49091D502907F64
:1011F00081E0903E09F080E080FF08C081E08093AC
:10120000CE0204C09F5F90932C0287CF0E943407C8
:101210000E9449070F90DF91CF911F910F91089580
:101220008091CD028350823018F40E943407F8CFA9
:10123000089580915603882369F0909157039F5F2A
:101240009F3019F09093570302C0109257038150BA
:101250008093560308958F929F92AF92BF92CF9240
:10126000DF92EF92FF920F931F93CF93DF93CDB74F
:10127000DEB729970FB6F894DEBF0FBECDBF8C0145
:1012800020915803211104C0C8010E942E057EC080
:10129000FC01C480D580E680F7806091590370918D
:1012A0005A03FB0185919591A591B491C816D90671
:1012B000EA06FB0648F3215030E0822F022E000C94
:1012C000990B831B910937FD939597FD0196959591
:1012D0008795830FFB0199E08902E00DF11D112430
:1012E00085909590A590B4908C149D04AE04BF0495
:1012F00018F431E0380F07C0C814D904EA04FB041D
:1013000038F42FEF280F231724F08213D6CF01C013
:10131000282FE9E02E02600D711D112449E050E0F4
:10132000CE0101960E94890CF80191818F81911163
:1013300003C0813039F4A8CF913009F0A5CF8823BC
:1013400009F4A2CF2D813E8189819A81AB81BC8134
:10135000820F931FA11DB11DF8012085C20ED11C63
:10136000E11CF11C8C159D05AE05BF0508F48CCF62
:10137000E885F985309709F487CFB801CE01019649
:101380000995F8018081882309F47ECF29960FB64C
:10139000F894DEBF0FBECDBFDF91CF911F910F91AB
:1013A000FF90EF90DF90CF90BF90AF909F908F9085
:1013B0000895CF92DF92EF92FF920F931F93CF93F6
:1013C000DF93CDB7DEB7C954D1090FB6F894DEBFAD
:1013D0000FBECDBF80915603882309F460C0E09012
:1013E000570384E0E89E70011124D701A65EBC4F2C
:1013F0006D018D919C91892BF1F10E9466088823E3
:1014000009F44DC08E010F5F1F4F89E4F80111925E
:101410008A95E9F7D601ED91FC91C8010995C801BB
:101420000E943105882321F1F60111821082DB80B0
:101430000E940508D81218C0DC800E940508D91245
:1014400013C08981882319F0C8010E942B09F70174
:10145000E65EFC4FE280F3800E941909E114F1047A
:10146000F1F0C801F7011AC0C8010E94380817C07E
:101470000E94190914C0CE0101960E944B088823CE
:1014800071F0D60112960D911C9113970E941909C3
:101490000115110521F0CE010196F8010995C75BF0
:1014A000DF4F0FB6F894DEBF0FBECDBFDF91CF91F7
:1014B0001F910F91FF90EF90DF90CF9008959C01C6
:1014C00090E02115310581F0F90189E0989FE00D48
:1014D000F11D112445915591659174919F5F4C3F89
:1014E0005F4F6F4F710581F730935A032093590373
:1014F0009093580308950C9400080E9405080895DD
:101500000E946D0810925A031092590310925803CA
:1015100010925703109256030895CF93DF93CDB7DF
:10152000DEB7C954D1090FB6F894DEBF0FBECDBFE8
:101530000E947A08CE0101960E940A08882359F079
:101540008981882321F0CE0101960E942B09CE01CA
:1015500001960E9425080E94D909C75BDF4F0FB68C
:10156000F894DEBF0FBECDBFDF91CF9108950E94EA
:101570006608811105C00E94D9090E947A08F7CF38
:101580000C941009FC01608171818281938108951E
:10159000DC01FB0194818C91981B892F9181992307
:1015A00021F0913001F590E00EC0DB011996908595
:1015B000980F891739F0FA01E80FF11D20812D935A
:1015C0008F5FF7CF0895392F380F2085921758F481
:1015D000DF01A90FB11D19962C91DA01A30FB11DDE
:1015E0002C939F5FF0CF08950E9491040E94890B75
:1015F0000E94800A0E9497020E94D104882349F029
:101600000E94D8040E94E10B0E948D0A0E94B4023D
:10161000F3CF0E94B5020E94B70A0E947F0C0C947F
:10162000F4040C94D5030E94DA0310920601109280
:10163000050108950F931F93CF93DF931F92CDB7AA
:10164000DEB70AE010E0F801E95AFD4FE491E983C2
:1016500041E050E0B801CE0101960E94DA030F5F2D
:101660001F4F0834110579F71092060110920501F9
:101670000F90DF91CF911F910F910895CF93DF933A
:1016800000D000D0CDB7DEB744E050E0BE016F5FC0
:101690007F4F82E090E00E94D5038B8180959981F5
:1016A000891308C06C8160959A81691303C00E94F8
:1016B0000B0502C098E78FEF0F900F900F900F90DF
:1016C000DF91CF9108950F931F93CF93DF9300D0B5
:1016D00000D0CDB7DEB78C010E940D058983C8010B
:1016E0000E9410058A83998190959B8380958C83B5
:1016F00044E050E062E070E0CE0101960E94DA031F
:101700000F900F900F900F90DF91CF911F910F913D
:101710000895EF92FF920F931F93CF93DF9300D022
:10172000CDB7DEB72AE0E22EF12C0FEF1FEF41E03C
:1017300050E0BE016F5F7F4FC7010E94D5038981D2
:10174000082788E0A801569547959801217033270E
:1017500000FF02C028E034E88A01022713278150E5
:1017600089F72FEFE21AF20A88E4E816F104F9F695
:101770000F3F2FEF120711F400E010E042E050E0BD
:10178000BE016F5F7F4FC7010E94D50389819A8197
:1017900024E5E216F10439F022E0E20EF11C8F3F5D
:1017A0002FEF920759F38017910711F00E941A0B3F
:1017B0000F900F90DF91CF911F910F91FF90EF90BD
:1017C0000895EF92FF921F93CF93DF9300D000D044
:1017D0001F92CDB7DEB780910501909106018F3F32
:1017E0002FEF920709F480C041E050E0BE016B5F2B
:1017F0007F4F0A960E94D503209105013091060182
:101800002115310531F48FEF9FEF90935C038093A6
:101810005B034D8180915B0390915C03842748E0DA
:10182000FC01F695E795BC016170772780FF02C047
:1018300068E074E8CF0186279727415089F7909395
:101840005C0380935B032F5F3F4F2E33310529F0FC
:10185000309306012093050147C02FEF3FEF3093EF
:101860000601209305018F3F2FEF920719F09C830B
:101870008B8302C01C821B8210E098E4E92EF12CBD
:1018800042E050E0BE016F5F7F4FC7010E94D50369
:1018900089819A818F3F2FEF920731F422E0E20E87
:1018A000F11C1F5F173061F72B813C818217930772
:1018B000D9F08FEF9FEF9A83898342E050E0B70120
:1018C000CE0101960E94DA031F5F173008F010E086
:1018D000612F70E06C5D7F4F660F771F42E050E034
:1018E000CE0103960E94DA030F900F900F900F9095
:1018F0000F90DF91CF911F91FF90EF90089580910D
:10190000050190910601019619F00E94E10BF7CFB5
:101910000895FB01DC0102C005900D92415050403A
:10192000D8F70895DC01CB01FC01F999FECF06C080
:10193000F2BDE1BDF89A319600B40D92415050408D
:10194000B8F70895DC01A40FB51F4150504048F08E
:10195000CB01840F951F2E910E94B30C4150504033
:10196000D0F70895262FF999FECF92BD81BDF89A40
:10197000019700B4021639F01FBA20BD0FB6F894D3
:0C198000FA9AF99A0FBE0895F894FFCF70
:08198C00010302FFFFFFFF0051
:00000001FF
